:100000000068000000130000DF880000000000000E
:1000100000000000000000000000000000000000E0
:1000200078FFE4B8200118F6D8F99000007F007E30
:1000300007E4F0A3DFFCDEFA75817A0223BC121A12
:10004000C312208F9002117401F022022C9274AA24
:100050007583F5758255A574557583FA7582AAA5C1
:1000600074A57583F5758255A52200021E87904000
:100070007FE493FF64326003EF7002002253A87F95
:100080000080FD0219401210CF902EC27412F0743D
:100090000F121176E4F0A37402F022022C8FE7090C
:1000A000F608DFFA8046E709F208DFFA803E888228
:1000B0008C83E709F0A3DFFA8032E309F608DFFA60
:1000C0008078E309F208DFFA807088828C83E30984
:1000D000F0A3DFFA806489828A83E0A3F608DFFA5E
:1000E000805889828A83E0A3F208DFFA804C80D2AC
:1000F00080FA80C680D4806980F28033801080A628
:1001000080EA809A80A880DA80E280CA803389827F
:100110008A83ECFAE493A3C8C582C8CCC583CCF02B
:10012000A3C8C582C8CCC583CCDFE9DEE7800D89D2
:10013000828A83E493A3F608DFF9ECFAA9F0EDFBD9
:100140002289828A83ECFAE0A3C8C582C8CCC58321
:10015000CCF0A3C8C582C8CCC583CCDFEADEE8807A
:10016000DB89828A83E493A3F208DFF980CC88F0EC
:10017000EF60010E4E60C388F0ED2402B40400501D
:10018000B9F582EB2402B4040050AF232345822347
:100190009008CE73EF8DF0A4A8F0CF8CF0A428CEF9
:1001A0008DF0A42EFE22C2D5EC30E709B2D5E4C30F
:1001B0009DFDE49CFCEE30E715B2D5E4C39FFFE45F
:1001C0009EFE120BF2C3E49DFDE49CFC8003120B27
:1001D000F230D507C3E49FFFE49EFE22C5F0F8A3EA
:1001E000E028F0C5F0F8E582158270021583E0384A
:1001F000F022BB010A89828A83E0F5F0A3E0225055
:100200000687F009E71922BBFE07E3F5F009E319B9
:100210002289828A83E493F5F074019322BB01075B
:1002200089828A830209BC500B09C5F027F7C5F003
:100230001937F722BBFE0D09F8E325F0F3C5F019D5
:10024000E338F322F889828A8374019325F0C5F09C
:10025000F8E4933822BB010A89828A83F0E5F0A38F
:10026000F0225006F709A7F01922BBFE06F3E5F0CD
:1002700009F3192275F008758200EF2FFFEE33FEA7
:10028000CD33CDCC33CCC58233C5829BED9AEC996E
:10029000E58298400CF582EE9BFEED9AFDEC99FC10
:1002A0000FD5F0D6E4CEFBE4CDFAE4CCF9A8822257
:1002B000B800C1B90059BA002DEC8BF084CFCECD77
:1002C000FCE5F0CBF97818EF2FFFEE33FEED33FDB0
:1002D000EC33FCEB33FB10D703994004EB99FB0F95
:1002E000D8E5E4F9FA227818EF2FFFEE33FEED336C
:1002F000FDEC33FCC933C910D7059BE99A4007ECE4
:100300009BFCE99AF90FD8E0E4C9FAE4CCFB22752A
:10031000F010EF2FFFEE33FEED33FDCC33CCC833BE
:10032000C810D7079BEC9AE899400AED9BFDEC9A20
:10033000FCE899F80FD5F0DAE4CDFBE4CCFAE4C898
:10034000F922EB9FF5F0EA9E42F0E99D42F0EC6461
:1003500080C864809845F022EB9FF5F0EA9E42F059
:10036000E99D42F0E89C45F022E8600FECC313FCE5
:10037000ED13FDEE13FEEF13FFD8F122ECF0A3ED29
:10038000F0A3EEF0A3EFF022A8828583F0D083D013
:1003900082120B7F120B7F120B7F120B7FE473E430
:1003A00093A3C583C5F0C583C8C582C8F0A3C58320
:1003B000C5F0C583C8C582C822EC8EF0A4CCC5F0B8
:1003C000CCCDF8EFA4CEC5F02DFDE43CFCE8A42E86
:1003D000C8C5F03DFDE43CFCEFA4FFE5F028FEE4D9
:1003E0003DFDE43CFC22EF4E6012EF60010EEDBBE0
:1003F000010B89828A83F0A3DFFCDEFA2289F050A8
:1004000007F709DFFCA9F022BBFEFCF309DFFCA91A
:10041000F022BC000BBE0029EF8DF084FFADF0226E
:10042000E4CCF875F008EF2FFFEE33FEEC33FCEE72
:100430009DEC984005FCEE9DFE0FD5F0E9E4CEFD65
:1004400022EDF8F5F0EE8420D21CFEADF075F00838
:10045000EF2FFFED33FD4007985006D5F0F222C391
:1004600098FD0FD5F0EA22208A03020FD1900214E2
:10047000E07002A3E06003020FD1900171E070020E
:10048000A3E06003020FD11211606003020FD1904C
:100490000132E0703090011D120FE6FFAEF09001C6
:1004A0000B120FE6D39FE5F09E4003020FD112100E
:1004B00070E490017DF0A3F01211C29002181211A5
:1004C000D9F5758003757500757614E4F5B2F5BA43
:1004D000900181E0F55DA3E0F55EC209758D2043D2
:1004E0008D20758D8043AA08D2AF758B02758EAFB3
:1004F000200624121160701F200C1CE5DB20E2177F
:10050000758AC4200C0DE5DB20E208758703000026
:10051000008006D2098002D209758B11758A50536A
:10052000AAF7D3900213E09490900212E094014055
:100530000EA3E02470F0900212E034FEF08007E495
:10054000900212F0A3F0D390021FE0949090021E4C
:10055000E09401400EA3E02470F090021EE034FE0F
:10056000F08007E490021EF0A3F01229F8900055E5
:10057000E075F006A4902EC3F0A3E4F0A3F01210EF
:100580002353997F1208661210D9902EC0E030E2F2
:10059000F9902EC0E4F0902E02E0F577A3E0F57814
:1005A0004389021210294380021210D6902EC0E017
:1005B00030E2F91211EDF522A3E0F523E5782527C5
:1005C000FFE5773526FEC3EF9523F525EE9522F559
:1005D0002412119FE5259FE5249E40048E248F253B
:1005E000902EC4E4F043998090016FE524F0A3E5D8
:1005F00025F0C3E55E9525FFE55D9524FE122C7080
:100600008E5F8F601212004003020FAAAE24AF2546
:100610007C007D14120B9912120AAF74AE73AD7286
:10062000AC719002C4121009FBD3120B389002C4B3
:1006300040171211229574FFEE9573FEED9572FD31
:10064000EC9571FC12120A8007120B680000000082
:10065000E47F607EEAFDFC9002C4121009FBD31215
:100660000B38400A9002C4120B680000EA60120FB7
:10067000E37D091211849002C41210097B0A121042
:100680005E12120A900132E07042AE5DAF5EFC7DF8
:1006900009120B99C8ECC8C9EDC9CAEECACBEFCB99
:1006A000E4FCFDEB2525FFEA352412109DE47B0ACE
:1006B00012106A8E5D8F5E9002C4120FF4121058F1
:1006C000121109120FFE121058020FAA121109126C
:1006D0000FFE12105890010E120FE6FFAEF09002BE
:1006E000C4121006FBD3120B385003020FBA120FBC
:1006F000D2121159FEC3EF957AEE95795003020F8D
:10070000BA90010B120FE6FFAEF07C007D02120BD7
:1007100099C8ECC8EDC0E0EEC0E0EFC0E0120FD227
:10072000121159FEE4FCFDD0E0FBD0E0FAD0E0F974
:10073000EB2FFFEA3E12109DE47B0312106A90013A
:100740000B120FFE1210C890010B120FE6D394305B
:10075000E5F094754008747575F030120A35900113
:1007600084E06066121167406190010B120FE6127F
:100770001159FE122C709002C8EEF0A3EFF0900118
:100780000B120FE6FFC312104C50199002C9E094EF
:100790001E9002C8E09400400B120FFBF9E475F0C4
:1007A000051209FD900185E0602090010B120FE613
:1007B00012104A4015D39002C9E094289002C8E074
:1007C00094004006120FFB1211F720090D121200BF
:1007D00050081211607003020CBC900183E00412F7
:1007E00011371210149001337401F0900216121197
:1007F0008C2290010EE0FBA3E0FAA3E0F91209D2EB
:10080000FFAEF0900108E0FBA3E0FAA3E0F90209D3
:10081000D2900134A3A3E0F9A3E0FF90010EE0FB26
:10082000A3E0FAA3E022E4FCFDE0F8A3E0F9A3E0F2
:10083000FAA3E0227A0079667E007F0B7D007B00C0
:10084000020BC643AB025389FD5395FD5396FD221F
:10085000C8ECC8C9EDC9CAEECACBEFCBE0FEA3E035
:10086000FF22A3F0A37401F0A322D3FF900189E03B
:100870009F900188E095F022C98FF0020A352FFF82
:10088000EA3EFEE93DFDE83CFCE4FAF9F8020A9094
:100890007F087A0179347E007D007B01020BC6E57A
:1008A0000A25E02428F8E6FE08E622A3F0A3740354
:1008B000F0A374E8F022F9EB2FFFEA35F0FEED39F2
:1008C000FDEC38FC22A3E0FEA3E0FBCAEECAE4F98B
:1008D000F822902E427D14E0FEA3E0FF7C00020986
:1008E00074F9E4F5F0020A35F9EE8FF0020A35905A
:1008F0002EC07402F022122C5B902EC07419F022CC
:10090000E50D25E02475F582E43401F583E0FEA3CE
:10091000E0FF229002C6E0FEA3E0FF2290018AE001
:10092000FCA3E0FDC3EF9DFF229002C4A3A3E0F966
:10093000A3E0FF900108229002147402F0A37458FF
:10094000F022E0FCA3E0FDA3E0FEA3E022900186FC
:10095000F0A3F0A3F0A322F07E007F057D007B00D2
:100960007A007961020BC6FFE5F0F0A3EFF022E414
:10097000F50EF50DF50CF50B22C39FFFE5F09E2259
:1009800090001BE0642022900188E0FEA3E0FFD3EA
:100990009400EE940022902ECAF0902EC77401F0BD
:1009A000902EC422FFAEF07C00020B99E4F0A374F9
:1009B000C8F022AB0EAA0DA90CA80BD3020B38E588
:1009C000272488FFE5263413FED32290016FE56CBF
:1009D000F0A3E56DF02225E02428F8A60F08A61064
:1009E00022E490021AF0A3F022F9746175F0A802D3
:1009F0000A3590003A7410F022F0A3F0900220F033
:100A0000A3F022FEEF2401FFE43EC31322902EC088
:100A1000E4F0902E1EE022F974FF75F0FB0209FD50
:100A2000C3E5609576E55F9575229002C4020B5C84
:100A3000120FD2FDACF0D39FEC9E403490010E1209
:100A40000FE6FFC3ED9FFFEC95F0FED3EF9430EE81
:100A50009475400D9002C67475F0A37430F00212C4
:100A600093120FDD1211599002C6F0A3EFF08043EC
:100A7000120FE3FFAEF090010E120FE6FDACF0C3D3
:100A80009FFFEC9EFED3EF9410EE9427400C900253
:100A9000C674D8F0A374F0F08012120FE3FFC3ED18
:100AA0009FFEEC95F09002C6F0A3CEF0E49002C653
:100AB000F0A3F0900132E060501210F3D39400EEF6
:100AC00064809480401A900120120FE6FDD3EF9DC0
:100AD000EE95F0400B900218E4F0A37464F0801BD4
:100AE000D3900219E09400900218E09400400C901A
:100AF000010B120FE69002C6121147D20B90021E94
:100B0000740FF0A374A0F0800D90021C12108E7A66
:100B1000007952121018D39002C7E094009002C6D8
:100B2000E06480948050030213E2E0F9A3E0FF90B8
:100B3000010B120FFE1210581210F3EE3395E0FD68
:100B4000FCE47BB87A88F9F8C3120B22500A9002B1
:100B5000C67488F0A374B8F0D390021BE0940090A0
:100B6000021AE09400500790001BE0B4201D121000
:100B7000F3C39496EE648094805010EF9400EE647A
:100B800080948040257C007D0A801430001C121067
:100B9000F3C394A0EE6480948F500F7C007D3212DA
:100BA00009869002C6EEF0A3EFF0900132E06031CA
:100BB00090021CE07002A3E07027900114120FE66F
:100BC0007D0F1211849002C6121030EE3395E0FDB5
:100BD000FCEB7B1012105E900114120FFEF9EE80F8
:100BE0000F9002C6E0F9A3E0FF900114120FFEC9B6
:100BF0008FF0120A35900114120FE624A8FFE5F0D9
:100C0000801D90010B120FFE1210C1900114120FE3
:100C1000FE1210C19002C7E024A8FF9002C6E03483
:100C200061F9900111120FFE1210582290018C12DE
:100C30001009FBE9C0E0EAC0E0EBC0E0900123123C
:100C40000FE6FFE4FCFDD0E0FBD0E0FAD0E01210AC
:100C50009690018C120B5C900191E004F07006906C
:100C60000190E004F0900192E07002A3E0600302C2
:100C700015D490018C121122FFEEC0E0EFC0E012FB
:100C800010A5D0E0FFD0E0FE120A9090018C120B6C
:100C90005C90018CA3A3E0FFA3E090018ACFF0A3B6
:100CA000EFF0A3120B6800000000E4900190121115
:100CB0003074C8F0900212E07002A3E060030215E5
:100CC000D4900132E07003021566900186E0FEA325
:100CD000E0FF4E702290018AE0FDA3E0900186CDF6
:100CE000F0A3EDF090010B120FE6FD900188E5F006
:100CF000F0A3EDF002154F1210FCEE9CFE122C70CA
:100D0000900198120FFE1210C8900184E070269096
:100D10000198120FE6C39412E5F09400500F900171
:100D20000B120FE6FF900188121148802090018479
:100D30007401F08018900198120FE6C39402E5F058
:100D400094005009E412112DF0900184F090018A72
:100D5000E0FEA3E0FFD3900187E09F900186E09E34
:100D60004007E4900185F080069001857401F0E46D
:100D7000900194F0A3F090019EF090019B120FFE61
:100D80001210C10215D4900194E0FEA3E0FF4E7052
:100D90001290018AE0FDA3E0900194CDF0ED1210D5
:100DA0008B80511210FCEE9CFE122C7090019B1255
:100DB0000FFE1210C8900196E07002A3E07035900B
:100DC000019B120FE6D39419E5F09400400C9001BA
:100DD000967413F0A37488F0800BE490019EF09059
:100DE000019612108E90018AE0FFA3E0900194CF4B
:100DF000F0A3EFF0900132E0700812112DF0900195
:100E000084F0221210CF902EC4E4F0A3F053997F07
:100E1000F50BF50CF50DF50EF50A12086612102308
:100E20001210D9902EC0E030E2F9902EC0E4F043C9
:100E30008902121029438002902E02E0FEA3E025D1
:100E40000CF50CEE350BF50B1210D6902EC0E030E1
:100E5000E2F91211EDFEA3E0250EF50EEE350DF5CB
:100E60000D050AE50AC3940640B0439980902EC54B
:100E7000E4F0E527240CFFE52634FEFED3EF950CC5
:100E8000EE950B4015900171E07002A3E070129096
:100E9000017104F0A374F4F08007E4900171F0A3F1
:100EA000F0E50C2527FFE50B3526FEC3EF950EF583
:100EB00010EE950DF50F12119FE5109FE50F9E4066
:100EC000048E0F8F10900167E50FF0A3E510F090EE
:100ED000016BE50DF0A3E50EF0A3E50BF0A3E50C27
:100EE000F0AF10AE0F1222CD90016FEEF0A3EFF035
:100EF00090001BE0B4200312101490016FE0FEA3D9
:100F0000E0FFE4FCFDE5692FF569E5683EF568ED75
:100F10003567F567EC3566F566056BE56B700205C0
:100F20006AC3E56F94E8E56E9403402AAE6AAF6B3E
:100F3000CBEFCB1210ABAF69AE68AD67AC66120AEF
:100F4000908E6C8F6DE4F569F568F567F566F56A66
:100F5000F56BF56EF56FD3E56D9400E56C9400408C
:100F600059900170E0956DFF90016FE0956CFE90D7
:100F700002CAF0A3EFF0D394F9EE6480947F401599
:100F8000E094079002CAE06480948050081211AB8C
:100F9000E4F57080259002CAE0FEA3E0FF122C70F9
:100FA000D3EF9414EE648094804003757003E57071
:100FB000C3940350051211AB057090016FE0F5501A
:100FC000A3E0F55178287C007D007B007A00792A27
:100FD0007E007F2802094E900132E070030218540F
:100FE00012107090021612108E900184E0700302AD
:100FF000193F121167500302193F90010B120FE6BF
:10100000121159FE122C709002C6EEF0A3EFF0D32D
:101010009496EE9400400CE4900184F0900186F0E8
:10102000A3F022900185E0602090010B120FE612E0
:10103000104A4015D39002C7E094289002C6E0946D
:10104000004006120FFB1211F790010B120FE6C3BE
:1010500012104B400302193F9002C7E0941E900209
:10106000C6E09400500302193F120FFBF9E475F03B
:10107000050209FD900134121009FBE9C0E0EAC045
:10108000E0EBC0E0120FE3FFE4FCFDD0E0FBD0E0BA
:10109000FAD0E0121096900134120B5C900139E006
:1010A00004F07006900138E004F0900216E070023F
:1010B000A3E0600302193F900134121122FFEEC039
:1010C000E0EFC0E01210A5D0E0FFD0E0FE120A90E1
:1010D000900134120B5C90010E120FE6241EFFE407
:1010E00035F0FE900134121006FBD3120B38403F4E
:1010F000900212E07002A3E0703590019EE0702F24
:10110000200B2C90013BE004F0700690013AE004C3
:10111000F0D390013BE0940590013AE09400401E2A
:10112000120FF1121058E490013AF0A3F0800F1260
:101130000FF1121058E490013AF0A3F0C20B9001A5
:1011400034120B6800000000E4900138F0A3F09026
:10115000019EE0900216600412118C2212108E2261
:10116000C0E0C083C082C0D0D2AF900225E004F0BE
:10117000D3900213E09400900212E09400400CA37C
:10118000E024FFF0900212E034FFF0D3900215E06B
:101190009400900214E09400400CA3E024FFF0902F
:1011A0000214E034FFF0D3900217E094009002168E
:1011B000E09400400CA3E024FFF0900216E034FF1E
:1011C000F0D3900219E09400900218E09400400CD3
:1011D000A3E024FFF0900218E034FFF0D390021B4C
:1011E000E0940090021AE09400400CA3E024FFF089
:1011F00090021AE034FFF0D3900223E094009002B2
:1012000022E09400400CA3E024FFF0900222E0349E
:10121000FFF0D3900221E09400900220E09400407F
:101220000CA3E024FFF0900220E034FFF0D3900202
:101230001DE0940090021CE09400400CA3E024FF09
:10124000F090021CE034FFF0C3E56F94E8E56E9483
:10125000035008056FE56F7002056EC3E55B94E807
:10126000E55A94035008055BE55B7002055AD3907C
:101270000193E09400900192E09400400CA3E024DC
:10128000FFF0900192E034FFF0D3900197E09400DA
:10129000900196E09400400CA3E024FFF0900196AA
:1012A000E034FFF0D3900172E09401900171E0947A
:1012B00000400CA3E024FFF0900171E034FFF0D374
:1012C00090021FE0940090021EE09400400CA3E006
:1012D00024FFF090021EE034FFF0D0D0D082D08303
:1012E000D0E0327E007FFF7D007B017A007904121E
:1012F0000BC69002D87400F0A37404F09001C5747A
:1013000001F0A37400F0A374B8F09001CB7401F065
:10131000A37400F074AC1229E57400F0A37494F087
:101320009001C87401F0A37400F0A374C6F090019A
:10133000D17401F0A37400F074D21229E57400F0A6
:10134000A3741F1229E67401F0A37402F0902DE03B
:10135000E493FF9002D8E0FCA3E0FDF5828C83A328
:10136000EFF0900002E0FFED24041229BF9000018D
:10137000E0FFED24051229BF900003E0FFED2406F5
:101380001229BF902DE2E493FFED24121229BF90A1
:101390002DE3E493FFED24141229BF9001DA7401C8
:1013A000F0A37400F0A3743CF0E4FF75F002EFA426
:1013B0002401F582E5F0342EF583E493FE74542F76
:1013C000F582E43400F583EEF0EF25E0242DF5827C
:1013D000E4342EF583E493FE1229EDEEF01229EDAC
:1013E000E0FEEF25E0242CF582E4342EF583E4932F
:1013F00024C0F582E4342EF583EEF00FEFB416AB83
:10140000902F56E0900058F0902F56E090006EF02C
:10141000902F56E0900059F0902F56E090006FF01A
:101420009000FF7401F09000FEF090003A7410F00C
:1014300090001BF0900028F0A37420F0900212742A
:1014400013F0A37488F02212114FF515F5168528B4
:1014500011852912852813852914F50A12107FFF9A
:10146000D3E5149FE5139E40078E138F14850A164B
:10147000C3E5129FE5119E50078E118F12850A1544
:10148000050AE50AB414D5E4F50FF510F50AE516DA
:10149000650A602EE515650A6028E510450F701095
:1014A000E50A25E02428F8E6F50F08E6F510801295
:1014B00012107F2510FFE50F3E1211E3F50FEF1319
:1014C000F510050AE50AB414C5900181E50FF0A3F3
:1014D000E510F0E516C394115005E5161211B6E5B6
:1014E00015C394115005E5151211B612114FF50AE6
:1014F00012107FFFC3E5109FFFE50F9EFE122C70B8
:10150000D3EF9419EE64809480400FE4FCFDE50E67
:101510002510F50EE50D350F800F12107FFFE4FC4E
:10152000FDE50E2FF50EE50D3EF50DED350CF50C38
:10153000EC350BF50B050AE50AC3941440B2AF7401
:10154000AE73AD72AC71121193401AE50E9574F53D
:101550000EE50D9573F50DE50C9572F50CE50B9503
:1015600071F50B800312114FE47F607EEAFDFC12DF
:101570001193400BE4750E60750DEAF50CF50BAE9A
:101580000DAF0E2290017DE0FEA3E0FFC39404EEB8
:101590009400502F900106E0FCA3E0FDEF25E0FF52
:1015A000EE33FE74752FF58274013EF583ECF0A3E3
:1015B000EDF090017EE004F0700690017DE004F013
:1015C000021E29750D011210E0E50D25E02473F5CA
:1015D00082E43401F583EEF0A3EFF0050DE50DB4E0
:1015E00004E4120FE3FF9001061210FFE5F09CFEE9
:1015F000122C70C3EF9428EE64809480503C9001CC
:1016000032E0702890010E120FE6FFC3900107E050
:101610009FFF900106E095F0FE122C70C3EF94142A
:10162000EE64809480500590010E800390010812B2
:101630000FE6FF90017BE5F0800B900106E0FFA331
:10164000E090017BCFF0A3EFF0E4F50CF50BF50A89
:10165000F509F50DD390017EE0950D90017DE094A4
:1016600000401E1210E0E4FCFDE50C2FF50CE50B2C
:101670003EF50BED350AF50AEC3509F509050D8047
:10168000D3AF0CAE0BAD0AAC09EEC0E0EFC0E090FA
:10169000017D1210A6D0E0FFD0E0FE120A908F0C60
:1016A0008E0B8D0A8C0922C0E0C083C082C0D0ECB2
:1016B000C0E0EDC0E0EEC0E0EFC0E0D2AFE5DB306F
:1016C000E419D20CC208E5DB30E102802E9002D78B
:1016D000E5DFF09002DAE4F0021F85E5DB30E50F8C
:1016E000D206300805C208021F85C20C021F85C23F
:1016F00008E5DB30E13AE5DB30E0109002DBE0FFAB
:1017000004F0122C45E0F5DF021F859002DBE0FFBC
:10171000B40813208A10D28A9002D8E0FCA3E024F7
:1017200007122C4BE4F0EF641A707AD207021F857F
:101730009002DAE0700EA3E5DFF09002DA7401F0B7
:10174000D20880619002DBE0902A6A93FFB4FF0820
:101750009002D7E5DFF08047EF640F70299002DB3D
:10176000E0FFA3E0FCA3E0FD122C4AE0540FF09050
:1017700002DBE0FF04F0ED122C4AE0FFE5DF54F05D
:10178000FEEF4EF0801F9002DBE0FF122C45E5DFFC
:10179000F0EFB4240A9002147401F0A374F4F090F2
:1017A00002DBE004F075DBFFD0E0FFD0E0FED0E02C
:1017B000FDD0E0FCD0D0D082D083D0E0329002CAFD
:1017C000EFF09002CFE4F0A374FFF0E4A3F0A3F0F5
:1017D000A304F0A374FFF0902EC07402F0902EC307
:1017E0007408F0E49002CBF0A3F09002CBE0FEA3EB
:1017F000E0FFC39409EE9400400302208CEF9407AD
:10180000EE940040067E007F0180199002CBA3E099
:1018100004FFE47E01C8EFC8088006CEA2E713CE1D
:1018200013D8F8FF9002CDEEF0A3EFF0902EC07425
:1018300019F0902EC0E030E2F99002CAE0FF75F096
:1018400002A424001229D4E0FCA3E0FD902EC07471
:1018500002F0D3ED94FFEC940F40179002CDE0FC22
:10186000A3E0FD75F002EF1229D1EC8DF01209BC56
:1018700080299002CAE075F0021229D1C083C0828B
:10188000E0FEA3E0FF9002CDE0FCA3E0FDC3EF9DEE
:10189000FFEE9CD082D083F0A3EFF09002CCE00466
:1018A000F070069002CBE004F0021FCA7F00227F96
:1018B000997A0179061210769001087401F0A374E8
:1018C00000F074441210427400F074461210427416
:1018D00000F0A374481210437400F0A37432121085
:1018E000437400F0A3742E1210437400F0A3742C00
:1018F000F09001237401F0A37400F0A37426F0901B
:1019000001987401F0A37400F0A37484121043745E
:1019100000F0A37486F09001267401F0A37400F027
:10192000A3741C1210437400F0A37422F090011AE7
:101930007401F0A37400F0A374361210437400F025
:10194000A3742A1210437400F0A37438F075790060
:10195000757AC890011A120FFEF9E579857AF012AE
:101960000A3590011D120FFEF9E475F064120A3574
:10197000900120120FFEF9E475F096020A359002EC
:10198000C6EEF0A3EF1211379002C6E07002A3E09A
:1019900060031222161226EBE490017DF0A3F07F83
:1019A00014122AA09002147402F0745812108B9032
:1019B0000106E0F9A3E0FFA3120FFE1210589001F8
:1019C0000B120FFE1210C1900111120FFE1211C95D
:1019D000900114120FFE1210C1900117120FFE1287
:1019E00011C91211D2E4900132F0900134120B6847
:1019F00000000000E4900138121130F0900106124E
:101A00000FF6121058E4900133F09002221211D90F
:101A100090021EF0A3F0FE7F14FD7B017A01798411
:101A2000120BC6900123120FE690018A1211479003
:101A3000019212118C22122B52902E42E0FEA3E052
:101A400024C4FFEE34FE9002C8F0A3EFF01210237E
:101A500053997F1229F81208661210CF902EC314E2
:101A6000F01210D9902EC0E030E2F9902EC0E4F0D0
:101A7000902E027D121210B78E268F277D14120B26
:101A800099EF24E0F574EE34B1F573ED34FFF5729F
:101A9000EC34FFF571438902121029438002439907
:101AA0008053997F122C5B902E5EE4F0A374FFF0BC
:101AB0007F0F121F9D902E5EE0FEA3E0D394F0EE08
:101AC00094014007902E5EE4F0A3F0902EC4E4F061
:101AD000439980A3F0900105E0900021F01210B22C
:101AE000900126120FFEF9EE8FF0020A359002CC1B
:101AF000EEF0A3EFF0E5644563700C9002CCE0F5E6
:101B000063A3E0F56480169002CDE02564FF9002A7
:101B1000CCE035631211E3F563EF13F5640565E579
:101B200065D3940A400D856361856462E4F563F5CD
:101B300064F565D3E5629400E5619400405A900233
:101B4000CDE09562FF9002CCE09561FE122C70C34F
:101B5000EF940AEE648094805026AE61AF627C0000
:101B60007D03120B999002CC121030E4FCFDEB2F98
:101B7000FFEA3E12109D7802120B499002CC8013AE
:101B80009002CDE02562FF9002CCE03561C313FEE8
:101B9000EF13FFEEF0A3EFF09002CCE0FEA3E0FF26
:101BA00022022AFBE493A3F8E493A34003F6800106
:101BB000F208DFF48029E493A3F85407240CC8C387
:101BC00033C4540F4420C8834004F456800146F6C1
:101BD000DFE4800B0102040810204080902571E4AE
:101BE0007E019360BCA3FF543F30E509541FFEE41F
:101BF00093A360010ECF54C025E060A840B8E493E1
:101C0000A3FAE493A3F8E493A3C8C582C8CAC58322
:101C1000CAF0A3C8C582C8CAC583CADFE9DEE780A7
:101C2000BE30000875791B757A5880067579007585
:101C30007AC890010B120FE6FFAEF0C3957AEE95CD
:101C4000795015900132E06020900120120FE6FDDE
:101C5000C3EF9DEE95F0401190021AE07002A3E0F0
:101C6000702790013204F0802090001BE0B4200522
:101C70001211C1800690021A12118CE4900132F008
:101C8000900218F0A3F01211D2900132E06011908E
:101C90000028E090003AB410047410F0227420F090
:101CA0002290022FE014601B1460432402705D90A8
:101CB0000239E0B4010A90022F1224EDD205D200BD
:101CC000C203227F02122902EF60077F02122C7CDE
:101CD000C205900239E0703490022F7402F0D203F2
:101CE000C205C2007F03122C7C7F0302279D7F0365
:101CF000122902EF60167F03122C7C900239E090CB
:101D0000022F7003F080031224EDC203227401F04D
:101D10007F02122C7C7F0212279D22CDEFCD43AD96
:101D2000105399EF439A10539BEF902EC07402F01A
:101D3000147E00C8EDC8088005C333CE33CED8F971
:101D4000FF902EC4EEF0A3EFF0902EC8EEF0A3EFBC
:101D5000F07410122BAE902EC0E030E2F9902EC03D
:101D6000E4F07402F07420122BAE902EC0E030E24A
:101D7000F9902E00E0FEA3E0FF902EC4E4F0A3F063
:101D8000902EC0F0439910539AEF539BEF5390EF6E
:101D900022C10C41023300410234004102300041B3
:101DA000023800C102C101C1044102390041022FC1
:101DB00000C103C100C1054102DA004102DB00425B
:101DC00002D50000C106C108C1074102D710410178
:101DD000030041010510C10BC10A41019F00022609
:101DE00000000471000000004101041041023A00AB
:101DF000009002C47408F0A3E4F0A3743FF0A3744D
:101E0000DFF0E4FDFCF9758A10538AEF009002C4FC
:101E1000E0FEA3E02DF582EE3CF583E493FF69F943
:101E20000DBD00010CBC37E5BDDFE29002C6122CEF
:101E300052E493699002D87009122C52A37413F0E3
:101E40008006122C52A3E4F0758A50538AEF0022C8
:101E5000200A06200303300509E4FFFE12215EC2BA
:101E60000A22900220E07002A3E060051211607067
:101E70003A200003122A311226EB7F01122AA01207
:101E80001D649002C4EEF0A3EFF07B017A0279C4E6
:101E90001228369002C412110E120FFE12105812A0
:101EA000121012240112140C1217B7122984229056
:101EB0000211E024FE6013146023146027240370D1
:101EC000499002117402F0122C8B7F017E001221C6
:101ED0005E9002117403F0E4900230F0229002113F
:101EE0007404F0221224811227EE122481900171D1
:101EF000E07004A3E06401700C900171F0A3F09015
:101F000002117402F0E4900225F0224389025395F5
:101F1000FD5396FD438002122BE87F0C1224FBCA6E
:101F2000EECACBEFCB7F0C1224FBEF2BFFEE3A90E7
:101F300002C9F0A3EFF0122BBAF91209D245F070E2
:101F400006122B9FEE80181209D2FBAAF0122B9FCB
:101F5000EF2BFFEE3AC313F9EF13FF122BBAC98F21
:101F6000F0120A35221229DDF5828E83A3E0B4AA8D
:101F7000031225D11229DDFF1229C8E0B41008EFA1
:101F80001229C8E4F0D20A1229DDFF241B1229CA43
:101F9000E0700DEF241C1229CAE0B4100312287D52
:101FA0001229DD24131229CAE0FFB4100690023969
:101FB0007401F0EFB42005E4900239F0229002C4DD
:101FC000EFF0E024BB122BC8E060037F01229002F7
:101FD000C4E0FF24BB122BC87401F0EF122BD0E435
:101FE00093FE740193FFE4FCFD902F60E0F8A3E002
:101FF000F9A3E0FAA3E02FFFEA3EFEED39EC3890BA
:1020000002C4E0122BDCEEF0A3EFF07F00221211ED
:1020100060702990019FE0700312111790019F7466
:1020200001F0900029E0B42008122630120C4780FD
:1020300003122ACE9002247401F08017E490019FCD
:10204000F0900029E0B42003122630900224E060D2
:1020500002E4F0022C0B9002C6EBF0A3EAF0A3E935
:10206000F0900214E07002A3E07031900133E06060
:102070002BE4900133F01226EB1211177508017F43
:1020800001122AA0121D649002C6120FFE1210C87F
:102090000508E508C3941440E61211C12212082E67
:1020A000E4F5F275F30875EEFF75EF3F75EA81F51B
:1020B000F675EB0700E5EC30E7FBE4F5EC9002D8B1
:1020C000E0FEA3E0FF241BF582E43EF583E5F3F098
:1020D000EF241CF582E43EF583E5F2F075EB302247
:1020E000758B11902F647440F0E4FEE4FFEF75F0FF
:1020F00003A4244DF582E43402F583E5822EF582B3
:10210000E43583F583E4F00FEFB40AE10EEEB40397
:10211000DA7F099002BBE4F0A3DFFC902F647480A7
:10212000F022CBEFCB122BC5E06036902F60A3A33B
:10213000E0FEA3E0FFEB122BDCE0FCA3E0FDD39F6D
:10214000EC9E501DC3EF9DFFEE9CFEEB122BD0C307
:102150007401939FE4939E4008122BC5E4F07F0125
:10216000227F0022758A50538AEF9000027411F08A
:102170009000017422F09000037433F0E4F5AB7525
:10218000AC1DF5ADF5AF7589FF75913F7599FFF5FC
:102190009675931CF59BF595F592F59A5388FCD2AC
:1021A0008AD20D2290003AE0FC900104E06C602E8F
:1021B00090003AE0FE900104F090000BE0900238AD
:1021C000F0540FF0EEB42005E04420800AECB41087
:1021D0000B900238E04410F090000BF0C28A22F518
:1021E00082E43CF583EFF022241AF582E43EF58385
:1021F00022A42440F582E5F0342EF583229002D803
:10220000E0FEA3E022A3F0A37401F0A322746A2FDE
:10221000F582E43400F583221210CF902EC4E4F04E
:10222000A3F0FF74542FF582E43400F583E0FE75CB
:10223000F002EFA42400F582E5F0342EF583E49358
:1022400024C0F582E4342EF583EEF00FEFB416D3FC
:1022500022300735C207902E42E0FFA3E09002C66D
:10226000CFF0A3EFF0122B521210B2900126120FF2
:10227000FE1210C81210CF9002C6E0FFA3E0902E0D
:1022800042CFF0A3EFF01211172200000000FFFF71
:10229000FFFF0000FFFFFFFFFFFFFFFFFF00FF004A
:1022A0000000FFFF000000FFFFFFFFFFFFFF000037
:1022B0000000FFFFFFFFFFFFFFFFFFFF0000000028
:1022C0009002C9EFF01229F8E4F5099002C9E0FF85
:1022D000E509C39F50071215E3050980EE902EC053
:1022E000E4F0121C27900106EEF0A3EFF022E4F5D3
:1022F000B2F5BA758D20438D20538D7F53AAF7F523
:102300008BE5DB20E211200C0EE4F58A75870300D3
:102310000000758A50D20A758B112212084E53A8FC
:102320007F12294412081E122B2743A880122C85E5
:102330009000FFE060069002117401F0122C291247
:10234000274512268F80F59002D8E0FFA3E0900287
:10235000DCCFF0A3EFF0E4F5DA75DA4043DA20756C
:10236000D74075DA5875D90143A90875B80875F8CA
:10237000082212102353997F1229F8902E42E4F07C
:10238000A374FFF01208667F01121F9D4389021299
:1023900010294380024399802201F400280028017B
:1023A000F4009603E801F403E81770006403E80002
:1023B0003202580258012C01F403E8271000C8909B
:1023C00002C9E0FEA3E0FF7C007D14020974902E98
:1023D000C2F0902EC0E04419F022900123E0FBA34C
:1023E000E0FAA3E02274BB2BF582E43402F58322E9
:1023F00025E0248DF582E4342BF5832225E0243B6F
:10240000F582E43402F58322902EC07402F0902EFF
:10241000C77474F0902ECD74C0F0A374FFF0A3F0D5
:10242000902EC37401F0902ECAF022E5B230E00580
:10243000E5AA20E013E4900226F075B28E75B6F995
:10244000F5B743B20143AA0122E4FF300616900219
:10245000D8E0FCA3E0F5828C83E0FE54F0FFEE545C
:102460000FF0C20622A3E0FCA3E02FF582E43CF5C6
:102470008322E0FEA3E0F5828E83221210CF902EFD
:10248000C27412F074091211767480F0A3E4F02281
:10249000EE30E707C3E49FFFE49EFE2274BB2F12D9
:1024A0002BC8E4F022122C950228C01211D222D29D
:1024B000AF32D2AF32022C0B00000000000000004F
:1024C000000000000000000000000000000000000C
:1024D00000000000000000000000000000000000FC
:1024E00000000000000000000000000000000000EC
:1024F00000000000000000000000000000000000DC
:1025000000000000000000000000000000000000CB
:1025100000000000000000000000000000000000BB
:1025200000000000000000000000000000000000AB
:10253000000000000000000000000000000000009B
:10254000000000000000000000000000000000008B
:10255000000000000000000000000000000000007B
:10256000000000000000000000000000000000006B
:10257000000000000000000000000000000000005B
:10258000000000000000000000000000000000004B
:10259000000000000000000000000000000000003B
:1025A000000000000000000000000000000000002B
:1025B000000000000000000000000000000000001B
:1025C000000000000000000000000000000000000B
:1025D00000000000000000000000000000000000FB
:1025E00000000000000000000000000000000000EB
:1025F00000000000000000000000000000000000DB
:102600001303AB68000000000000000000000000A1
:1026100000000000000000000000000000000000BA
:10262000021203030A0F0DA00EB60FFF0C020BFFE0
:1026300023F724062504070127082A0828022B026D
:1026400029032C032D082E082F0426080211030647
:102650000A100D400E800FFF0C020BFF23F4240420
:102660002504070127102A1028042B0429032C0312
:102670002D202E202F10262000000000000000003A
:10268000000000000000000000000000000000004A
:10269000000000000000000000000000000000003A
:1026A000000000000000000000000000000000002A
:1026B000000000000000000000000000000000001A
:1037F0000000000000000000000000000000003B8E
:1038000000000000000000000000000000000000B8
:1038100000000000000000000000000000000000A8
:00000001FF
